:0E00000084C1FECFFDCFFCCFFBCFFACFF9CFEE
:10000E00F8CF1EC309C2F5CFB4C1F3CFF2CFF1CFF3
:10001E00F0CFEFCFEECFEDCF20204144534C205404
:10002E004553544552202020000020202020762EBB
:10003E00332E302E352E20202020000050A9A8204F
:10004E0022A045A75445A7454B4F4D220000AA2D8F
:10005E00A720224DA154432220E14F5450200000EE
:10006E0042C3B26570B8BF65207065B6B8BC3A00C1
:10007E00416E6E65782D412020416E6E65782D4261
:10008E00000020205061B77061B26FBFC0B8BA3A9D
:10009E00202000002020AAB8BBB8BE6FB3B8C02085
:1000AE00412EA52E00002020A86FE3BABBC6C06566
:1000BE00BDB86520BA2000006365BFB82E2E2E2075
:1000CE00A3E3B8BF652E2E2E000020A16FBF6FB325
:1000DE0020BA207061B26FBF6500205065B6B8BC03
:1000EE003A2000002043B8B4BD61BB2FAC79BC20D0
:1000FE0020202020000020A461BF797861BDB86562
:10010E002020202020200000204D61BA632E206385
:10011E00BA6F706F63BFC4200000205465BA79E6D1
:10012E002E2063BA6F706F63BFC40000204D6FE660
:10013E00BD6F63BFC420BE657065E32E0000202036
:10014E00050520202020000020200607202020204A
:10015E000000202020202020202000002F0020E062
:10016E006F2063B3B8E361BDB8C72E2E2E200000FA
:10017E0020736F6B6F6C2E75636F7A2E636F6D20AD
:10018E00000020E3A02E2020202020202020000090
:10019E0020E3A0BC2E20202020202020000020BA0A
:1001AE00B22F632E20202020200001010101010129
:1001BE000300FF01010101010300FFFF0101010125
:1001CE000300FFFFFF0101010300FFFFFFFF01011D
:1001DE000300FFFFFFFFFF010300FFFFFFFFFFFF15
:1001EE0003000202020202020400FF0202020202E5
:1001FE000400FFFF020202020400FFFFFF020202E0
:10020E000400FFFFFFFF02020400FFFFFFFFFF02DB
:10021E000400FFFFFFFFFFFF04006164736C2069A1
:10022E006E666F202D2D73686F770000010101013E
:10023E00010101011F00000000000000000000008D
:10024E000000001F10101010101E1E1E1E1E1E106D
:10025E0010101010000004040404041F0707070305
:10026E00010101011C1C1C18101010101027E803AE
:10027E0064000A00010000100001100001000000DF
:10028E008813960000000041050020204572726F11
:10029E007223202530357520200020416E7376653F
:1002AE007223202530357520200020556261742080
:1002BE003D2025692C253032752056202020002027
:1002CE0055636867203D2025692C253032752056F0
:1002DE002020200080C0010002008C02020061027A
:1002EE008E02010068029002040086029202010052
:1002FE00DA0296020200DB02E2020000F894EE2718
:10030E00ECBBF1E0FBBFEBBFE5BFF8E1F1BDE1BD3A
:10031E008DE0A2E0BB27ED938A95E9F780E094E0AB
:10032E00A0E6ED930197E9F7E4EEF2E08591959161
:10033E00009761F0A591B59105901590BF01F00160
:10034E0005900D920197E1F7FB01F0CFEFE5EDBFC0
:10035E00E4E0EEBFC0E6D1E026C4E881E066E7B98E
:10036E0085E28A95F1F7369A349BFECF349AE5B141
:10037E0099C7EA93FA93EFB7EA930DDD1BB10CB16F
:10038E00E12FEC7179F4E52D53941FD90083EFEF33
:10039E00E51509F455247394EFEFE71519F4772456
:1003AE00689420F802DDE991EFBFF991E991189573
:1003BE001A93A8957720F1F3A895E42D439405D9C7
:1003CE001081EFEFE41509F44424F8947A947894AC
:1003DE00E12F1DC3FED8E5E0E3BFF894E6E9E09314
:1003EE00680278940895E0E0E3BFF3D808954424BA
:1003FE00F894772444245524E89420F878940895AA
:10040E00EBD8EAD800D9E8ECF0E000D9F0DF01D95A
:10041E00FDD802D907D9089509D9DBD8E091680231
:10042E00E03031F0E0916802E150E093680201C0E3
:10043E000BD925C2B0DCEA81EE0FEE0FEE0FE064B1
:10044E000E2F10E0183060F40A930395EC81FD81B5
:10045E003196EC83FD83FCD8EA93ACD61F5FF2CFC6
:10046E005AC7E881F981F695E795DF01E881F981B0
:10047E00E170F07008DCE070F47BEA27FB27ABC676
:10048E0024971A93E0E0E983EA83EB83EC8310E090
:10049E00123360F4E6E0DFD8E2D801DC01DB3ADBB0
:1004AE00E983FA836B837C831F5FF2CFDDD8D7D8C5
:1004BE0081DBBFDAE0936E02F0936F02DED8A73ACB
:1004CE00E4E0BE0710F0E6E024C0D7D8AE38E4E092
:1004DE00BE0710F0E5E01DC0D0D8A537E4E0BE079A
:1004EE0010F0E4E016C0C9D8AC35E4E0BE0710F059
:1004FE00E3E00FC0C2D8A334E4E0BE0710F0E2E0A0
:10050E0008C0BBD8AA32E4E0BE0710F0E1E001C09B
:10051E00E0E0E0937202E0E0B5D81881FDC61A93D0
:10052E00E0E0E0937002E093710210E0193038F4CD
:10053E00E5E091D8AAD8AED8B0D81F5FF7CFA5D82E
:10054E00E7E0F0E0BEDBA9D862C2E0E0E0935F0234
:10055E00879B03C0A7D8E160A8D8B09B03C0A2D8E0
:10056E00E260A3D89FD8E030B1F4E0E0E093D80287
:10057E00A0916B02A13070F0A0916B02AE3148F4E5
:10058E00E0936B02E0936D02E0916002E0936C02E7
:10059E00089528C027C0E0916002A0915F02EA177B
:1005AE00F1F4E0916B02EF5FE0936B02A0916B02AE
:1005BE00AE3108F40895E091D802EF5FE093D802CF
:1005CE00A091D802AB3048F06DD8E0936C02E1E018
:1005DE00E0936D02E0E0E093D802089507C062D880
:1005EE00E0936002E0E0E0936B0208950895D3DBA0
:1005FE0000E010E01A3020F4B2990F5F1F5FFACFBF
:10060E00073018F00093850203C0E0E0E093850206
:10061E00CCDB0895BEDB20E030E010E01A3030F481
:10062E00E5E019D82E0F3F1F1F5FF8CFD901EAE082
:10063E00F0E047DB9F0120938402B2DB24960895FD
:10064E00F5D73CD8A0916902A33021F4A0916502A0
:10065E00A53008F00EC0A091D902AF5FA093D902C9
:10066E00A43639F4E0E0E093D902B4DEC0DED4D78C
:10067E00D9D7A091DA02AF5FA093DA02AA30D1F5F2
:10068E00E0E0E093DA02E1E0FDD7B1DF1CD899F0AB
:10069E00939AA0918402AB3710F419D850F0A0E0D1
:1006AE009499A1E0E1E0EA2711F4949801C0949A9C
:1006BE0001C0949814C0A0917202A23058F4949A7A
:1006CE00A0E09399A1E0E1E0EA2711F4939801C02C
:1006DE00939A02C093989498FFD708F402D8A091E9
:1006EE007402A63020F4E0917402EF5F01C0E0E0E6
:1006FE00E0937402A0916902A03021F0A0918502CE
:10070E00A03009F00BC0A1E6B2E0F4D7E09161028F
:10071E00F0916202309709F4E4D706C0E8E8F3E1FD
:10072E00E0936102F093620210DFE0916D02E0301F
:10073E0059F1E0916902E03059F4E2D7A13011F499
:10074E00E1E0E1D7DDD7A33011F4EFEFDCD71BC02A
:10075E00DED7C8F0A0916902AF3F09F4DBD7C1D74D
:10076E00E0917902F0917A02A0917B02B0917C0225
:10077E00EA17FB0741F4EEEFE0938302E091830268
:10078E00A2E0B0E0F3DA76C0CAD7CDD761F4CFD706
:10079E0011F4D0D7969ABBD729F4E2E0E0936A021F
:1007AE00B2D7959A67C0CBD7C1F4C1D751F4A091F7
:1007BE006502A43018F4C7D7EF5F01C0E0E0E09304
:1007CE006502A5D749F4BFD7E03019F0BCD7E15088
:1007DE0001C0E4E0E09365024DC0E83CA0E0FA07FA
:1007EE00F9F4A5D779F4B2D7A081A93048F4A09135
:1007FE007D02B2D7A258BD4FEC91EF5FEC9302C0D1
:10080E00A5D7ACD784D759F4A0917D02A43020F49B
:10081E00E0917D02EF5F01C0E0E0E0937D022AC02F
:10082E00EF3FA0E0FA0731F582D791F49AD7A2D71D
:10083E0006DA09F008F403C0A2D765D901C0A5D71E
:10084E00E0938602F0938702609388027093890288
:10085E005ED781F486D799D7F2D918F490D75AD9A2
:10086E0001C088D7E0938602F093870260938802D6
:10087E0070938902E0E0E0936C02E0936D02E991DF
:10088E00EFBFF991E991B991A991999189917991D6
:10089E006991F9901990099018957CD77FD711F42A
:1008AE0083D7FCCF85D787D779D711F090D7FCCFD8
:1008BE0092C470D779D772D711F476D7FCCF87D779
:1008CE006DD711F084D7FCCF82D772D7A881B981AA
:1008DE0080D7E0D680D7A0837EC41A93E3E0E715D5
:1008EE0008F095C0A89560D776D7A33509F08FC0CC
:1008FE00E42D6BD6A081AE3409F089C06FD7A23536
:10090E0009F085C010E0173030F46ED7E657FD4F72
:10091E0025D71F5FF8CF6AD76ED7173030F464D75C
:10092E00EF56FD4F1BD71F5FF8CF68D764D7173030
:10093E0030F45AD7E856FD4F11D71F5FF8CF34D792
:10094E004AD7A13419F030D7A895FACF5CD753D730
:10095E00173030F449D7E156FD4F00D71F5FF8CF5F
:10096E0057D749D7173030F43FD7EA55FD4FF6D653
:10097E001F5FF8CF19D72FD7A03519F015D7A89527
:10098E00FACF4BD738D7173030F42ED7E355FD4F6B
:10099E00E5D61F5FF8CF46D72ED7173030F424D7C1
:1009AE00EC54FD4FDBD61F5FF8CFFED614D7AD3417
:1009BE0019F0FAD6A895FACF3AD76FDF10E01730B4
:1009CE0030F412D7E554FD4FC9D61F5FF8CF34D798
:1009DE0064DF10E0173030F407D7EE53FD4FBED66C
:1009EE001F5FF8CFE1D6F7D6A23519F0DDD6A89560
:1009FE00FACF27D752DF10E0173030F4F5D6E75391
:100A0E00FD4FACD61F5FF8CF21D747DF1DD619910A
:100A1E000895E3E0E71518F5C7D6DDD6AD34F9F441
:100A2E00E42DD3D5A081AF36D1F4D8D6A436B9F4FF
:100A3E00B1D6BAD6D0D6AA3311F0B6D6FBCFB4D62D
:100A4E00E0916602EA937DD3E03011F0ADD6F8CF97
:100A5E0002D7C1D6AD3011F0FED6FBCFF5D5089535
:100A6E00E3E0E715C8F4A0D6B6D6AE36A9F4E42D69
:100A7E00ACD5A081A53681F4B1D6A33669F4E42DA8
:100A8E00A8D6EE59FE4FA081A43731F4E0E0E093F2
:100A9E006302E1E0E09364020895E8D6E7D691D3CD
:100AAE00E5D6ABD3E3D6E5D68CD3E0D6A6D3E88194
:100ABE0090D6309759F4DDD6D9D683D3E8EBF1E052
:100ACE00DBD6D7D67ED3E0EFF1E04FC02CD659F46B
:100ADE00D0D6CCD676D3E0ECF1E0CED6CAD671D352
:100AEE00E8EFF1E042C0CCD659F4C3D6BFD669D3F5
:100AFE00E8ECF1E0C1D6BDD664D3E0E0F2E035C05B
:100B0E001ED659F4B6D6B2D65CD3E0EDF1E0B4D62B
:100B1E00B0D657D3E8E0F2E028C0E430A0E0FA0700
:100B2E0059F4A7D6A3D64DD3E8EDF1E0A5D6A1D6BC
:100B3E0048D3E0E1F2E019C0E530A0E0FA0759F43D
:100B4E0098D694D63ED3E0EEF1E096D692D639D32F
:100B5E00E8E1F2E00AC08DD689D633D3E8EEF1E0B3
:100B6E008BD687D62ED3E0E2F2E0FA93EA9365D3E2
:100B7E0099C33DDD85DCE1E085D5A895A4D589F442
:100B8E00ABD568F473D689DFA8957ED6A8957CD6AA
:100B9E00A89523D379D6A89577D6A89501C00895A0
:100BAE0001C00895E6CF6197F894E0E0E8BBE2E07B
:100BBE00E7BBE4E0E2BBE8E7E1BBE0E0E5BBE3BBBB
:100BCE00E3BF07D57BD5E3E0EEBDE5E0E9BFE0E0AE
:100BDE00EBB9E8E9EAB9E6E0E0BDE0E0E0BDE5E06A
:100BEE00E9B9E7E6E7B9E6EDE6B9E9E3E1BDE9E241
:100BFE00E1BDA895E4E1EA9329D3A895EAE3F2E0F2
:100C0E0046D634D617DCE2E4F2E041D632D612DC18
:100C1E00EAE4F2E03CD6E2E03DD6E2E5F2E037D699
:100C2E00E3E038D6EAE5F2E032D6E4E033D6E2E6A7
:100C3E00F2E02DD6E5E02ED6EAE6F2E028D6E6E0A2
:100C4E0029D6E2E7F2E023D6E7E024D6A895A0E085
:100C5E00B0E06CD8EF77F070E0937502F093760207
:100C6E00A2E0B0E067D8E0938302A3E0B0E05AD8E8
:100C7E0013D677D58AD5E3D711F008F004C071D515
:100C8E0079D5DDD728F4E0E0F0E060E071E404D639
:100C9E0041D5A3D2EBD5EAD594D2E6E2F0E005D663
:100CAE00E5D5E7D58ED2E8E3F0E0FFD5A895ECD5F3
:100CBE00A895EAD5A895E8D5A8958FD25ADF78944D
:100CCE00D5D5D4D57ED2EAE4F0E0EFD5CFD5D1D5C7
:100CDE0078D2ECE5F0E0E9D5A895D6D5A895D4D58F
:100CEE00A895D2D5A89579D2C1D5C0D56AD2E0E95A
:100CFE00F0E0DBD5BBD5BDD564D2E2EAF0E0D5D5C8
:100D0E00BFDBE1E0BFD4BA9AE5E0F0E07FD4BA9859
:100D1E00A895BAD5A895B8D5A895B6D5A895FFDB50
:100D2E00E0917002F0917102A8D4EA2BFB2BAFD5A3
:100D3E0098DBE0937702F0937802B9D5A8D591DBD2
:100D4E00E0937902F0937A0248D2E0917202EA932C
:100D5E00A4DEA895E4D4309731F5B5D441F4A89526
:100D6E0093D5A89591D5A8958FD5A8951BC0A09180
:100D7E008402AB3710F4ABD418F0E091740202C0C9
:100D8E00E0917202EA9389DEE8E0EA936FD519D218
:100D9E00ECE4F1E08AD5E8E0EA936BD512D2E6E511
:100DAE00F1E083D5BEC1BFD401F5A0917502B0911B
:100DBE007602109721F4A0918302AE3F99F48299A6
:100DCE000DC054D553D5FDD1EEE6F0E06ED54ED51F
:100DDE0050D5F7D1EEE7F0E068D503C0ABD4969AC4
:100DEE00959A02C0E8EC8FD49CC14AD571F53ED5D8
:100DFE003DD5E7D1E4EBF0E058D538D53AD5E1D181
:100E0E00E6ECF0E052D50ED4E0E0E093640254D567
:100E1E0019F026DEA895FBCFE0916402E030A1F038
:100E2E00DCD100D4EDDA48D519F0F3DDA895FBCF6F
:100E3E00F9D342D519F051DDA895FBCFE3E0E0934D
:100E4E006902E5E0E09365026CC179D409F0E5C072
:100E5E00A0916502A53091F409D508D5B2D1E8ED7F
:100E6E00F0E023D503D505D5ACD1E8EEF0E01DD5E5
:100E7E00E0EDF2E025D5E0E6F1E017D5E09168026D
:100E8E00E03009F064C0EDE2E093A602E0939F0229
:100E9E00E0939802E0939102E0938A02E093AD0210
:100EAE00E093C902E093C202E093BB02E093B40266
:100EBE00E093A702E093A002E0939902E0939202DE
:100ECE00E0938B02E093AE02E093CA02E093C3027A
:100EDE00E093BC02E093B50212E01730C0F584D463
:100EEE000F01DF01E657FD4FFF93EF93FD01EF5624
:100EFE00FD4FCF01F001E856FD4FBF0175D4E1560D
:100F0E00FD4F0F01A12F28D4AA55BD4FDBD4AF91B1
:100F1E00BF91EC9369D40F01DF01EC54FD4FFF93A9
:100F2E00EF93FD01E554FD4FCF01F001EE53FD4F60
:100F3E00BF015AD4E753FD4F0F01A12F0DD4A35576
:100F4E00BD4FC0D4AF91BF91EC931F5FC6CFFBD303
:100F5E0040D4309781F48AD489D433D1E6E1F1E0DC
:100F6E00A4D484D486D42DD162D4B5D465D458D12A
:100F7E00ECEAF1E049C0D7D381F478D477D421D10B
:100F8E00E8E2F1E092D472D474D41BD15AD4A3D433
:100F9E005DD446D1ECEAF1E037C072D481F466D468
:100FAE0065D40FD1E2EFF0E080D460D462D409D1E1
:100FBE001DD491D423D434D1E0E9F1E025C0BFD3C0
:100FCE0081F454D453D4FDD0E4E0F1E06ED44ED489
:100FDE0050D4F7D018D47FD41BD422D1E0E9F1E05D
:100FEE0013C0E430A0E0FA0791F440D43FD4E9D026
:100FFE00EAE3F1E05AD43AD43CD4E3D00ED46BD425
:10100E0011D40ED1EEE9F1E0FA93EA9316D154D44D
:10101E0019F063DCA895FBCF84C0E83CA0E0FA078A
:10102E00A9F560917E027727A0917F02EAE057D45E
:10103E00A0918002E4E653D4A09181028DD3E8EE14
:10104E00F3E03AD66E0F7F1FA091820285D3E0E1C6
:10105E00F7E232D6E60FF71FE0937B02F0937C02A5
:10106E0043D415D4E8E9F2E012D421D43FD4FED310
:10107E0044D43AD40CD4E8EAF2E009D4E0917B02ED
:10108E00F0917C0233D4F5D338D44BC0EF3FA0E0BF
:10109E00FA07C1F444DA28D4FAD3E8EBF2E0F7D336
:1010AE00ECD22ED4EAD232D4E1D327D41DD4EFD34E
:1010BE00EDECF2E0ECD3E9D223D4E7D227D4D9D3A6
:1010CE001CD42FC0EA30A0E0FA0759F5FCD299F4EF
:1010DE00CDD3CCD376D0ECE6F1E0E7D3C7D3C9D3EA
:1010EE0070D0EEE7F1E0E1D3A895CED3A895CCD39E
:1010FE00A895CAD3A89513D4309719F0A5E7B2E0F6
:10110E00F9D20DD4A0E0B0E029D6C1989598969862
:10111E00E0E0E0936402E0936302E0936902E093FF
:10112E006A02E0917302E03011F0AAD973DA11CE9F
:10113E00FFCFE1E0F991F03310F0FA3308F0EE272B
:10114E000895E1E0F991F03229F0F93010F0FE3017
:10115E0008F0EE270895E881E07111F0A89A01C019
:10116E00A898E881E07211F0A99A01C0A998E881C7
:10117E00E07411F0AA9A01C0AA98E881E07811F003
:10118E00AB9A01C0AB9887E08A95F1F7C59A82E1D8
:10119E008A95F1F7C59882E18A95F1F783C0E881C7
:1011AE00C3D3E881E295E883E881BED388EB8A95C4
:1011BE00F1F778C0E981BAD3C49AE881B7D3C4985D
:1011CE000AC0E88106D3E552FD4FE081A981EA0FFE
:1011DE00ADD36980988022960895E2E0A7D3E3E02C
:1011EE00F0E014D2ECE0A2D344D3D9DFE3E0F0E098
:1011FE000DD2E0E09E2E6E2E0895A881AA3011F039
:10120E00681440F033D393949A92DBDFA881AA300E
:10121E0009F448C06394C49AE88188D3C49842C044
:10122E001A93A981BA81ED91A983BA831E2FE0305A
:10123E0019F01A93E2DFF5CF42C01A9379D31E2F1D
:10124E00E03019F01A93D9DFF9CF39C0A09AA19ADC
:10125E00A29AA39ABD9ABC9ABB9AC598C498C398F1
:10126E008880E881E058E093DD02E881E054E09365
:10127E00DE02E4E1F0E0CAD1E0E356D35FD35ED301
:10128E0063D3E0E251D360D3E8E250D3E4E04ED32F
:10129E00E5E84CD3E6E04AD3A0DF04C05D9BFECF69
:1012AE00E881ECB9219608951A9342D31E2FE030AF
:1012BE0019F01A93F3DFF9CFEAE0EA93EFDF188122
:1012CE002396089568D545D312961FD53097F1F021
:1012DE0040D342D38F01309761F00230E0E01E0719
:1012EE00A0F0F80131978F01AA81BB811496ED937E
:1012FE00FC932FD3129633D33197AC81A08329D38D
:10130E0004D5FF2312F025D32AD305C022D3EFEF45
:10131E00FFEFED93FC9346D525960895269737D586
:10132E0010E0AC85BD85E0E0F0E0ED93FC93EA893A
:10133E00FB893196EA8BFB8B8BD12E2FE03009F493
:10134E00FEC0E12FE03031F4253211F411E001C07E
:10135E000CD3F4C0E130A1F4253211F406D3EDC064
:10136E0012E040E000E02D3211F401E0E7C02B3234
:10137E0011F44BE2E3C0203211F440E2DFC002C0B0
:10138E00E23039F450E013E0203311F40068D6C097
:10139E0003C0E33009F0D2C0203310F02A3308F036
:1013AE0007C0AAE05A9F502DE22FE0535E0FC6C031
:1013BE00E22FE33639F4E1D2E3D2DFD2A481AA934D
:1013CE00E3D2BBC0E33731F4E6D2E7D2E9D2E8D0BC
:1013DE001E2F08C0E03751F4DED2DFD2E1D2EAD0C0
:1013EE001E2F086002600F7730E02EC0E43611F039
:1013FE00E93611F4046002C0E53729F4EAE7F2E0B9
:10140E00D2D215E00BC0E83511F4086003C0E837FE
:10141E0009F093C0E4E8F2E0C6D214E002FF11C076
:10142E00BAD2BBD2C3D2AB85AA232AF4EA85FB85F6
:10143E002AD4BCD24DE2403011F01F5F01C00B7FA9
:10144E0003C0A9D2AAD2B2D200FD10C0151770F4F3
:10145E0007FF08C002FF04C00B7F242F115001C0EC
:10146E0020E301C020E281D25150F0CF312F01FF95
:10147E0015C0303091F003FF05C0EE81FF8125913C
:10148E0092D205C0AE81BF812D91AE83BF836DD246
:10149E00503009F051503150ECCF46C020E3EE8170
:1014AE00FF8137D4E887F987EE81FF8132967BD2B0
:1014BE00E885F985AA85BB85AE17BF0748F02F5F73
:1014CE00A885B985EA85FB85EA1BFB0B6FD2F0CFA9
:1014DE002A3328F003FF02C0295F01C0295D04FDF5
:1014EE0019C0213320F4A885B985119709F409C0D4
:1014FE00531710F000FF01C011C020E207FF0AC011
:10150E0020E3006102FF06C00B7F4A933DD25030AC
:10151E0009F051502AD2503009F051503150A8855F
:10152E00B985129708F0BACF00FF07C0503029F0E6
:10153E005150E0E2EA9328D2F9CF10E0F8CEAC8514
:10154E00BD85E3D32BD464960895FF92F82E26978B
:10155E0020D42FD2309719F4EFEFFFEF1DC0DE012C
:10156E0016968DD38D0125D21ED2E0E0E887E9874D
:10157E00DE011A9684D3C9D38AD11A930A93E9E667
:10158E00F9E085D1FE013A9682D1C8DE9F01AE8187
:10159E00BF81E0E0EC93F90103D42A96FF90089501
:1015AE00A991B991EE27FF276D91662311F031961F
:1015BE00FBCF0895AA27BB27E991F991059000204A
:1015CE0011F01196FBCFFD010895F0E0E05AFE4FA9
:1015DE000895E8E2E2BF0895EDE0EA935FDEE8ECFD
:1015EE00F0E0FA93EA93EAD1E1E6EA9357DEE4E615
:1015FE00EA9354DEEDE6EA9351DEE9E6EA934EDE37
:10160E00EEE6EA934BCEEDE0EA9348CEFA93EA93F8
:10161E00D5C1E4E6F0E00895E8E2F2E0FA93EA9349
:10162E0043DEF1CFE1E0E093630208950A921A924D
:10163E00FA926A937A938A939A93AA93BA93EA93B5
:10164E00FA93EFB7EA930895E0E0E0936302CBC616
:10165E003197E4910895EA9380D6F0E00895A98138
:10166E00BA818B819C810895E0918602F091870268
:10167E0060918802709189020895A0916E02B091D6
:10168E006F020895E09373020895A0917002B091D5
:10169E0071020895EA0FFB1F0895E0937002F09314
:1016AE0071020895E0915F020895E0935F02E8E809
:1016BE00F3E1E0936102F09362020895E0E8FCEB3F
:1016CE00FDBDECBD0895E0918502E0300895D5DFB3
:1016DE00A43FE4E0BE070895D0DFAB31E4E0BE07DF
:1016EE000895EAE0E0936902E0E0E0936402E0939B
:1016FE0063020895ED91FD913197FE93EE93089557
:10170E00A0916C020895E0936902C19A0895F8DFE2
:10171E00A2300895A9DFA3E0B0E018D30895E091B8
:10172E006902F0E00895E130A0E0FA070895E8DFDD
:10173E00A1300895E1E0E0936A02E2E0E4CFE33005
:10174E00A0E0FA070895E09165020895E0917D0208
:10175E00F0E0E258FD4F0895B0E00895A0E0A083B8
:10176E000895A0918602B09187028091880290918F
:10177E0089020895E0E0F0E060E771EC089574DF0F
:10178E00AFE6B2E183E09BE30895E0E0F0E060E7CE
:10179E0071E40895E0E0E09367020895E091660237
:1017AE00EA93C7DCE030089503D6E093660208950D
:1017BE00E09167020895A881B981F0E06BDFA091F6
:1017CE006602A083F5DFEF5FE0936702EDCFF0DFF7
:1017DE00F2CFF0E00895A09166020895E42DF9DFAE
:1017EE00EF59FE4FA0810895E12FF3CFEAE8F2E022
:1017FE00FA93EA9308955DD810E00895E1E9F2E0D6
:10180E00FA93EA930895E8E9F2E0FA93EA930895D9
:10181E00EFE9F2E0FA93EA930895E6EAF2E0FA933A
:10182E00EA930895EDEAF2E0FA93EA930895E4EB71
:10183E00F2E0FA93EA930895EBEBF2E0FA93EA936F
:10184E000895E2ECF2E0FA93EA930895E9ECF2E0FF
:10185E00FA93EA930895ACDFBCDFE053FD4FBBDF94
:10186E00A083A6DFEF5FE09367029ECFE0E0EA93EE
:10187E000895E1E0EA930895FA93EA93DEDCF9CF56
:10188E00E230A0E0FA070895E4EFF1E0BFCEFA935C
:10189E00EA930895EA93CEC5E0938602F093870209
:1018AE0060938802709389020895F1DFC6CCE091AF
:1018BE007702F09178020895E0916302E030089586
:1018CE00E6DFAECCE0E0EC93D001EC93DB01EC93E1
:1018DE00DC01EC930895A4DCEAE6F1E0E6CFEA9FA2
:1018EE00F0016E0F7F1F0895FE010895662777277A
:1018FE0014D284E02ADE2896B9CF63DCF5DFE0CF80
:10190E0088DEDFD16627772708D2089582DEECD1F4
:10191E006627772702D288E018DE2C96A7CFE091B3
:10192E007502F09176020895EA9315CCEA9337CCBE
:10193E00E981FA813196E983FA838ACE84E191E0D6
:10194E000197F1F7E0E3F0CF84E191E00197F1F731
:10195E000895AA81BB8108951496D7D10895ED916B
:10196E00FD913196FE93EE9308952A93ED85FE85B3
:10197E008EDFE989FA8909950895E889F98908952C
:10198E003497E88BF98B0895ED85FE8580DFE98924
:10199E00FA8909950895F1DFF3CFA889B989DCCFCB
:1019AE00EE83FF8374CFEE83FF830895EA87FB8770
:1019BE000895DE011C9663D1A8D10895E991F9919D
:1019CE00309639F08DEC9AE00197F1F7A8953197A2
:1019DE00C9F70895552342F4503811F4E0FF04C0BE
:1019EE003196691F791F6BF050E8572711F45F93FA
:1019FE00CFC05F3F31F0660F000C57956795752F7E
:101A0E0008955F9300200AF0CFC0C8C050E8192E89
:101A1E001522880F991F9527550F879550E8072E89
:101A2E000522660F771F7527550F679508956894E1
:101A3E0001C0E8945F93F2DF703818F07F3F08F42E
:101A4E00A7C056E1571BAAF4519558300EF45930E1
:101A5E0030F0EFEFFFEF6FEF7FE777F91AC07727E0
:101A6E005523B9F0EE0FFF1F661F771F5A95D1F75A
:101A7E0010C07727583028F0EF2FF62F672F5850C9
:101A8E00F9CF552331F076956795F795E7955A95E9
:101A9E00D1F700200AF4FBD05F910895689401C03D
:101AAE00E894309760407040B1F0002426F0772320
:101ABE0012F40094ECD0172E7EE1112032F07A95BC
:101ACE00EE0FFF1F661F111CF9CFEF2FF62F612DA2
:101ADE005F938ADF5F9108954F93AF01FD01DA01A5
:101AEE00AB01BC01CA01402D012C142E4F9108955B
:101AFE00EA0FFB1F681F0895E095F0956095EF5F64
:101B0E00FF4F6F4F08955F9381DF903871F150E86A
:101B1E00152604C05F937ADF903839F1703821F1C1
:101B2E00572F591B2BF112F4D7DFFACF583118F07B
:101B3E00AA27BB278827583028F0AB2FB82F882725
:101B4E005850F9CF552329F08695B795A7955A95F4
:101B5E00D9F7502D512572F0CBDF38F46795F795F4
:101B6E00E795739513F420C0B7DF3EDF5F910895BC
:101B7E00D8F7FBCFEA1BFB0B680B51F010F4009467
:101B8E00BBDF662392F3EE0FFF1F661F7A95CBF72E
:101B9E00EE27FF27662777275F910895EFEFFFEF78
:101BAE006FE77FEF5F910895EFEFFFEF6FE77FE74E
:101BBE005F9108955F932ADF703821F411200AF4A3
:101BCE00EDCFF2CF903809F4E3CF01240894970BB0
:101BDE001BF4D4F30020F3CF792F1F932F933F9351
:101BEE004F9311241127222733274427552790E29C
:101BFE00AE17BF078607410730F0AE1BBF0B860B33
:101C0E00410B089401C08894551F221F331F111CCD
:101C1E00AA1FBB1F881F441F9A9551F7F901612D0A
:101C2E004F913F912F911F91662332F0550FEE1F6A
:101C3E00FF1F661F7A9543F2CDDE5F9108959923BB
:101C4E009AF0772342F0971748F029F4AE17BF07A2
:101C5E00860720F031F0989488940895989408940B
:101C6E0008951894889408957723C2F7971798F3D8
:101C7E00A9F7EA17FB07680788F399F3ECCF00245E
:101C8E00AF0DB01D0895F195E195F0400895F095D2
:101C9E0060957095E195FF4F6F4F7F4F08956F2FB1
:101CAE00660F660B762F0895FA9FF02DEB9FF00DC1
:101CBE00EA9FE02DF10D08951AD0F6DF0EF4E3DF62
:101CCE0008950024112490E1AA0FBB1F001C111CC3
:101CDE000E1A1F0A18F40E0E1F1E01C0A1609A954F
:101CEE0099F7FD01D0010895ECDFFD010895E89408
:101CFE00F7FF02C0C8DF6894B7FF06C0A095B09585
:101D0E00119600F8039400FA0895ED91FC91119745
:101D1E0008950590F491E02D08957A936A93FA93BD
:101D2E00EA930895129602D0BF011297119602D02F
:101D3E00FE2F1197E199FECFFF93FFB7F894AEBB3C
:101D4E00BFBBE09AEDB3FFBFFF91089507D0129687
:101D5E000F01FB0103D0F0011297089507D01196E1
:101D6E00EF93EF2F03D0EF9111970895E19B02C0EF
:101D7E00A895FCCF9FB7F894AEBBBFBBE09A8DB3CE
:101D8E00E81719F0EDBBE29AE19A9FBF08955A93B6
:101D9E004A933A932A931A930A9308955D814C813C
:101DAE003B812A811981088108950991199108951D
:00000001FF
